:0200000480007A
:100000006F00C0006F20C02B6F20802B930000007A
:10001000130100009301000013020000930200008E
:100020001303000093030000130400009304000076
:10003000130500009305000013060000930600005E
:100040001307000093070000130800009308000046
:100050001309000093090000130A0000930A00002E
:10006000130B0000930B0000130C0000930C000016
:10007000130D0000930D0000130E0000930E0000FE
:10008000130F0000930F00009702000093820201FB
:10009000739052307350447497020000938202F7B9
:1000A0007390523017D100001301C1E3F32240F1E5
:1000B0009392C2003301510073100134EF20D0132A
:1000C000173500001305C5946F20407383328510E7
:1000D000739012148330850003310501833185014B
:1000E000033205028332850203330503833385031C
:1000F00003340504833485048335850503360506FA
:1001000083368506033705078337850703380508D7
:10011000833885080339050983398509033A050AB7
:10012000833A850A033B050B833B850B033C050C97
:10013000833C850C033D050D833D850D033E050E77
:10014000833E850E033F050F833F850F033505056D
:10015000730020107311011423341100233C31006B
:10016000233041022334510223386102233C7102BF
:1001700023308104233491042338A104233CB104A7
:100180002330C1062334D1062338E106233CF1068F
:10019000233001092334110923382109233C310973
:1001A0002330410B2334510B2338610B233C710B5B
:1001B0002330810D2334910D2338A10D233CB10D43
:1001C0002330C10F2334D10F2338E10F233CF10F2B
:1001D000F312011423385100F32200102330511080
:1001E000F322101423345110F32230142338511009
:1001F000F3222014233C5110130501006F20C03757
:1010000000000000000000000000000000000000E0
:1010100000000000000000000000000000000000D0
:1010200000000000000000000000000000000000C0
:1010300000000000000000000000000000000000B0
:081040000000000000000000A8
:10200000B367B500B3E7C70093F77700B306C50021
:10201000638407023386C50093070500637ED502FB
:1020200003C705009385150093871700A38FE7FE6C
:10203000E398C5FE67800000E37ED5FE93070500A8
:1020400003B70500938787009385850023BCE7FECF
:10205000E3E8D7FE6780000067800000130101FFFE
:10206000B367C500233081002334110093F7770054
:10207000130405003307C500638207026376E50099
:1020800093F5F50FEFF09FFD8330810013050400F9
:1020900003340100130101016780000093F5F50F7F
:1020A0009727000083B78786B385F502E37EE5FCBA
:1020B000930705009387870023BCB7FEE3ECE7FE98
:1020C0008330810013050400033401001301010172
:1020D0006780000083470500638E070093070500B3
:1020E00003C7170093871700E31C07FE3385A7403B
:1020F000678000001305000067800000834705002B
:10210000938515001305150003C7F5FF638A0700C3
:10211000E386E7FE1B8507003B05E540678000007E
:10212000130500006FF05FFFB367B50093F777000A
:10213000639E0702137886FF330805016378050361
:10214000930705006F000001938787009385850042
:1021500063F8070183B6070003B70500E386E6FED0
:102160003385A7403306A640138507003386C50094
:102170006F00400103C705008347F5FF93851500F5
:10218000639AE70013051500E396C5FE13050000EA
:10219000678000003B85E7406780000093070500EB
:1021A00003C705009387170093851500A38FE7FEEB
:1021B000E31807FE6780000003470500930600024E
:1021C000930705006318D70003C71700938717000C
:1021D000E30CD7FE9306D0026300D7069306B00245
:1021E0006300D70483C607009305000063820604DA
:1021F0001305000093871700131725001B8606FDA3
:1022000083C607003307A700131717003305E6003E
:10221000E39206FE638005023305A040678000005C
:1022200083C617009305000093871700E39206FC0E
:10223000130500006780000083C617009305100097
:1022400093871700E39606FA130500006FF09FFED0
:1022500083470500638007049305101017F7FFFFFD
:10226000130747DA93950503033607001305150096
:10227000B3E6B700630A060097F7FFFF23B407DC55
:1022800083370700E39A07FE2330D7008347050012
:10229000E39C07FC6780000017F7FFFF130787D652
:1022A00083370700638A070097F7FFFF23BC07D82F
:1022B00083370700E39A07FE2330A7006F00000072
:1022C000130101FF1305903423341100EFF0DFFCFC
:1022D000130101FE1306810093077101130890009A
:1022E0006F008000930707009376F50013870600C0
:1022F000930500036374D800930570053B07B7008E
:102300002380E700135545001387F7FFE31CF6FC15
:1023100083478100230C010063820704130510101A
:102320009306060017F7FFFF1307C7CD1315050324
:10233000833507009386160033E6A700638A0500FD
:1023400097F7FFFF23B007D083370700E39A07FE14
:1023500083C706002330C700E39C07FC130101027A
:1023600067800000130101FB9307100037F7FFFFA0
:102370002322F1002334110423308104233C9102F1
:10238000233821032334310323304103233C5101FB
:1023900023340100B306E500B7E7030063F6F6183F
:1023A0009359C5009384096017390000130989C542
:1023B00093973400B307F90083B707003374E5003F
:1023C0006396071017770000130747C4033A070006
:1023D00063000A1883378A009776000083B686C2A6
:1023E0002330F700638CD712130641009305810058
:1023F00013050400833A0A00EF00C0606310051063
:1024000093D6CA009396A60093E6F60193973400FC
:10241000B307F90013E7060C23B0E70073000412BA
:1024200097270000938707BE93994900B387370128
:1024300003B707006318071203370A00B705040043
:1024400023B0E70003378A0023B4E700F3A50510A3
:10245000B707E0FFB307F4003716000013070400C6
:102460003386C70003B3070083B8870003B80701AA
:1024700003B5870123306700233417012338070190
:10248000233CA7009387070213070702E39CC7FCBE
:102490007390051093973400B304F90023B0D4006F
:1024A000730004120F100000833081040334010410
:1024B000833481030339010383398102033A010222
:1024C000833A8101130101056780000013F70704B7
:1024D0006302070413F70708631207061307F000E7
:1024E00093E70708639CE50493943400B3049900D0
:1024F00023B0F400730004126FF01FFB83360A0050
:102500008337810093D6C6009396A600B3E6F60003
:102510006FF0DFEF93E707046FF01FFD9777000080
:1025200023B207AE6FF05FEC171500001305853E70
:10253000EFF01FD213053000EFF01FD61715000083
:102540001305C541EFF0DFD013053000EFF0DFD405
:102550001715000013050545EFF09FCF1305300058
:10256000EFF09FD31715000013054545EFF05FCE40
:1025700013053000EFF05FD2130101F82338810614
:10258000233C11062334910623302107233C3105D7
:10259000233841052334510523306105233C710361
:1025A00023388103233491032330A103233CB10159
:1025B00013040500EF0080446312050E8335841177
:1025C000930780006380F510930720006380F50671
:1025D000938745FF130710006376F7009307F00019
:1025E000639CF51E03350411EFF0DFD713050400DB
:1025F00003340107833081078334810603390106E0
:1026000083398105033A0105833A8104033B0104C0
:10261000833B8103033C0103833C8102033D0102B0
:10262000833D8101130101086FD05FAA0337841035
:1026300093773700639E0706EF0780007310300022
:102640000327070083A707006300F7061305101090
:1026500093071004971600009386463A17F7FFFF7A
:102660001307479A13150503833507009386160051
:1026700033E6A700638A050097F7FFFF23B4079CA2
:1026800083370700E39A07FE83C706002330C7009D
:10269000E39C07FC13053000EFF01FC01305040096
:1026A000EFD0DFA26FF09FF113051000EFF0DFBE57
:1026B000171500001305853EEFF09FB91305300094
:1026C000EFF09FBD83270405B7140000972A000090
:1026D000938A4A932334F100173D0000130D8D9225
:1026E000B70C0400370CE0FF177A0000130A8A9138
:1026F000977B0000938B8B9137FB030093D7C4002B
:102700001399470033872A0103370700630C070832
:102710009387076093973700B307FD0083B90700DD
:1027200093F709046380070AF3AD0C103384840126
:10273000371600009305040013850400EFF0DF9EB8
:102740006304050493F909086380090AB7160000B9
:102750001387040093070400B386D40003380700EE
:1027600003358700833507010336870123B007014E
:1027700023B4A70023B8B70023BCC7001307070280
:1027800093870702E31CD7FCB3872A0173900D10CF
:1027900003370A0023B00700630007022334F70061
:1027A0002330FA00B7170000B384F400E39864F50F
:1027B00003358100EFF05FAE2330FA0023B0FB0059
:1027C0006FF05FFE1715000013054526EFF05FA8B8
:1027D00013053000EFF05FAC171500001305852ED0
:1027E000EFF01FA76FF01FEB1715000013058527EB
:1027F000EFF01FA613053000EFF01FAAF32740F1FA
:10280000639A0718974700009387C77F130101ED6C
:1028100093D7C70023308112175800001308887E11
:10282000130405009397A700173500001305857D55
:10283000233411129356C5001357C80093E71700AD
:10284000972800009388087C1306F0FF233CF5FED0
:102850009396A6001317A700B707002093E616006B
:102860001367170093D5C8001313F6039387F70C6B
:10287000233CF8FE23B0D8002330E500B3E7650021
:102880007390071873270018639EE7141356B60059
:102890009307F0019702000093824201F3925230B5
:1028A0007310063B7390073A739052301308F0BFD1
:1028B0001318580197E7FFFF9387078AB38707012B
:1028C00073905710F3270034B387070173900714F0
:1028D000B7B700009B87071073902730B7E7010058
:1028E0009B870760739007307350403017270000B4
:1028F000130747B09307083EB3060701B307F70075
:10290000B7080800176600002332D67017230000AE
:10291000130343ED9766000023B6F66E9388F80321
:10292000930730001308080113D61700B386170168
:10293000B347F600B30507019396C6009397570077
:102940002330D7002334B70093F70702130707019A
:10295000B367F600E31AE3FC1306001293050000C8
:10296000130501009727000023BA07E6EFF00FEFE9
:10297000B70700803304F4001305010023348110ED
:10298000EFD0CFF48330811203340112130101130D
:102990006780000013071000B7A76301370608001F
:1029A0009387D7841306C6FF1315F7019316E70321
:1029B0006F00C0012F20070013D71700B3C7E7002F
:1029C0009397E703B3F7D700B3E7E70033F7C70000
:1029D00093F517003307A700E39E05FC03200700CB
:1029E0006FF09FFD171500001305C510EFF05F860F
:1029F00013053000EFF05F8A6780000013050000C8
:102A0000678000001305000067800000731030002D
:102A10009301A000B77524009B85D58A9395E500A6
:102A20009385D5C49395C5009385755E9395D50020
:102A3000938505EF13060000D38005F2530106F2DB
:102A400053802022530500E2B77324009B83D38A6E
:102A50009393E3009383D3C49393C3009383735EF0
:102A60009393D300938303EFE31275689301B0004F
:102A7000B77524009B85D58A9395E5009385D5C4C9
:102A80009395C5009385755E9395D500938505EF65
:102A90001306F0FFD38005F2530106F25380202283
:102AA000530500E2B77324FF9B83D38A9393E3001B
:102AB0009383D3C49393C3009383735E9393D300A0
:102AC000938303EFE31475629301C000B77524FF8D
:102AD0009B85D58A9395E5009385D5C49395C500CC
:102AE0009385755E9395D500938505EF13060000D9
:102AF000D38005F2530106F253802022530500E2F1
:102B0000B77324009B83D38A9393E3009383D3C446
:102B10009393C3009383735E9393D300938303EFE4
:102B2000E316755C9301D000B77524FF9B85D58AA9
:102B30009395E5009385D5C49395C5009385755EFF
:102B40009395D500938505EF1306F0FFD38005F22A
:102B5000530106F253802022530500E2B77324FF8D
:102B60009B83D38A9393E3009383D3C49393C3004B
:102B70009383735E9393D300938303EFE3187556A7
:102B800093014001B77524009B85D58A9395E50094
:102B90009385D5C49395C5009385755E9395D500AF
:102BA000938505EF13060000D38005F2530106F26A
:102BB00053902022530500E2B77324FF9B83D38AEE
:102BC0009393E3009383D3C49393C3009383735E7F
:102BD0009393D300938303EFE31A7550930150014D
:102BE000B77524009B85D58A9395E5009385D5C458
:102BF0009395C5009385755E9395D500938505EFF4
:102C00001306F0FFD38005F2530106F25390202201
:102C1000530500E2B77324009B83D38A9393E300A8
:102C20009383D3C49393C3009383735E9393D3002E
:102C3000938303EFE31C754A93016001B77524FF8A
:102C40009B85D58A9395E5009385D5C49395C5005A
:102C50009385755E9395D500938505EF1306000067
:102C6000D38005F2530106F253902022530500E26F
:102C7000B77324FF9B83D38A9393E3009383D3C4D6
:102C80009393C3009383735E9393D300938303EF73
:102C9000E31E754493017001B77524FF9B85D58AA7
:102CA0009395E5009385D5C49395C5009385755E8E
:102CB0009395D500938505EF1306F0FFD38005F2B9
:102CC000530106F253902022530500E2B77324000B
:102CD0009B83D38A9393E3009383D3C49393C300DA
:102CE0009383735E9393D300938303EFE310754054
:102CF0009301E001B77524009B85D58A9395E50083
:102D00009385D5C49395C5009385755E9395D5003D
:102D1000938505EF13060000D38005F2530106F2F8
:102D200053A02022530500E2B77324009B83D38A6B
:102D30009393E3009383D3C49393C3009383735E0D
:102D40009393D300938303EFE312753A9301F00159
:102D5000B77524009B85D58A9395E5009385D5C4E6
:102D60009395C5009385755E9395D500938505EF82
:102D70001306F0FFD38005F2530106F253A0202280
:102D8000530500E2B77324FF9B83D38A9393E30038
:102D90009383D3C49393C3009383735E9393D300BD
:102DA000938303EFE314753493010002B77524FF96
:102DB0009B85D58A9395E5009385D5C49395C500E9
:102DC0009385755E9395D500938505EF13060000F6
:102DD000D38005F2530106F253A02022530500E2EE
:102DE000B77324FF9B83D38A9393E3009383D3C465
:102DF0009393C3009383735E9393D300938303EF02
:102E0000E316752E93011002B77524FF9B85D58AB2
:102E10009395E5009385D5C49395C5009385755E1C
:102E20009395D500938505EF1306F0FFD38005F247
:102E3000530106F253A02022530500E2B773240089
:102E40009B83D38A9393E3009383D3C49393C30068
:102E50009383735E9393D300938303EFE3187528F2
:102E6000930180029B05100093956502938595F070
:102E70009395D500938555349395C50093858567C3
:102E800013060000D38005F2530106F25380202080
:102E9000530500E0B703C07FE31A75249301C0080F
:102EA0009B05100093956502938595F09395D50049
:102EB000938555349395C500938585671306000067
:102EC000D38005F2530106F253802020530500E21F
:102ED0009B03F0DF93936301E31A75209301900243
:102EE000B725E1FF9B8555349395C500938585678C
:102EF00013060000D38005F2530106F25380202010
:102F0000530500E0B703C07FE312751E9301D0089C
:102F1000B725E1FF9B8555349395C500938585675B
:102F200013060000D38005F2530106F253802020DF
:102F3000530500E29B03F0DF93936301E318751AD6
:102F40009301A0029B05100093956502938595F867
:102F50009395D500938555349395C50093858567E2
:102F600013060000D38005F2530106F2538020209F
:102F7000530500E0B703C07FE31A75169301E0081C
:102F80009B05100093956502938595F89395D50060
:102F9000938555349395C500938585671306000086
:102FA000D38005F2530106F253802020530500E23E
:102FB0009B03F0DF93936301E31A75129301B00250
:102FC000B725F1FF9B8555349395C500938585679B
:102FD00013060000D38005F2530106F2538020202F
:102FE000530500E0B75334129B838367E3107510D9
:102FF0009301F008B725F1FF9B8555349395C500E3
:103000009385856713060000D38005F2530106F20D
:1030100053802020530500E2B723F1FF9B835334F4
:103020009393C30093838367E312750C930120038A
:103030009B05100093956502938595F09395D500B7
:10304000938555349395C500938585671B061000BD
:103050001316F601D38005F2530106F253802020A7
:10306000530500E0B703C07FE312750893016009C0
:103070009B05100093956502938595F09395D50077
:10308000938555349395C500938585671B0610007D
:103090001316F601D38005F2530106F25380202067
:1030A000530500E29B03F0DF93936301E310750483
:1030B00093013003B725E1FF9B8555349395C500F7
:1030C000938585671B0610001316F601D38005F261
:1030D000530106F253802020530500E0B703C07F60
:1030E000E316750093017009B725E1FF9B85553400
:1030F0009395C500938585671B0610001316F6018E
:10310000D38005F2530106F253802020530500E2DC
:103110009B03F0DF93936301631A757C9301400373
:103120009B05100093956502938595F89395D500BE
:10313000938555349395C500938585671B061000CC
:103140001316F601D38005F2530106F253802020B6
:10315000530500E0B703C07F631A757893018009B7
:103160009B05100093956502938595F89395D5007E
:10317000938555349395C500938585671B0610008C
:103180001316F601D38005F2530106F25380202076
:10319000530500E29B03F0DF93936301631875749A
:1031A00093015003B725F1FF9B8555349395C500D6
:1031B000938585671B0610001316F601D38005F270
:1031C000530106F253802020530500E0B753341218
:1031D0009B838367631C757093019009B725F1FF8A
:1031E0009B8555349395C500938585671B06100014
:1031F0001316F601D38005F2530106F25380202006
:10320000530500E2B723F1FF9B8353349393C3002C
:1032100093838367631C756C9301C0039B05100047
:1032200093956502938595F09395D50093855534D4
:103230009395C5009385856737060080D38005F296
:10324000530106F253802020530500E0B703C0FF6E
:10325000631E75689301000A9B0510009395650233
:10326000938595F09395D500938555349395C50036
:103270009385856737060080D38005F2530106F2F7
:1032800053802020530500E2B703C0FF631075662A
:103290009301D003B725E1FF9B8555349395C50075
:1032A0009385856737060080D38005F2530106F2C7
:1032B00053802020530500E0B703C0FF63187562F8
:1032C0009301100AB725E1FF9B8555349395C500FE
:1032D0009385856737060080D38005F2530106F297
:1032E00053802020530500E2B703C0FF63107560D0
:1032F0009301E003B725F1FF9B8555349395C500F5
:103300009385856737060080D38005F2530106F266
:1033100053802020530500E0B75334929B8383678A
:103320006316755C9301200AB725F1FF9B85553420
:103330009395C5009385856737060080D38005F295
:10334000530106F253802020530500E2B753349214
:103350009B838367631C75589301F003B725F1FFC6
:103360009B8555349395C500938585671B06100092
:10337000131606021306F6FF1316F601D38005F2A4
:10338000530106F253802020530500E0B753341256
:103390009B838367631C75549301300AB725F1FF43
:1033A0009B8555349395C500938585671B06100052
:1033B000131606021306F6FF1316F601D38005F264
:1033C000530106F253802020530500E2B723F1FF9A
:1033D0009B8353349393C30093838367631875501F
:1033E00093016004B715F1FF9B8515119395C500F6
:1033F000938515113716F1FF1B0616111316C6001B
:1034000013061611D38005F2530106F253802022D1
:10341000532500A01305F5FF63140500530500E0D4
:10342000B71311119B8313116312754C9301A00AFA
:10343000B715F1FF9B8515119395C500938515115F
:103440003716F1FF1B0616111316C60013061611C8
:10345000D38005F2530106F253802022530500E287
:10346000B713F1FF9B8313119393C300938313113D
:10347000631E754693017004B715F1FF9B85151106
:103480009395C500938515111B061000131676023F
:10349000130616F11316C600130616111316C600EE
:1034A00013061611D38005F2530106F25380202231
:1034B000532500A01305050063140500530500E023
:1034C000B71311119B831311631275429301B00A54
:1034D000B715F1FF9B8515119395C50093851511BF
:1034E0001B06100013167602130616F11316C600FB
:1034F000130616111316C60013061611D38005F213
:10350000530106F253802022530500E29B03100072
:1035100093937302938313F19393C30093831311D3
:103520009393C300938313116312753C930180043A
:10353000B715F1FF9B8515119395C500938515115E
:10354000371611911B061611D38005F2530106F2AE
:1035500053802022532500A01305F5FF63140500B6
:10356000530500E0B71311119B83131163107538D5
:103570009301C00AB715F1FF9B8515119395C500FE
:1035800093851511371611911B061611D38005F27C
:10359000530106F253802022530500E2B713F1FFD6
:1035A0009B8313119393C30093831311631075349A
:1035B00093019004B715F1FF9B8515119395C500F4
:1035C000938515111B06F0FF1316F603D38005F241
:1035D000530106F253802022532500A01305F5FF66
:1035E00063140500530500E0B71311119B831311F9
:1035F000631E752E9301D00AB715F1FF9B85151137
:103600009395C500938515111B06F0FF1316F6035D
:10361000D38005F2530106F253802022530500E2C5
:10362000B713F1FF9B8313119393C300938313117B
:10363000631E752A9301A0049B05100093957502E3
:10364000938515F19395C500938515119395C50044
:10365000938515113716F1FF1B0616111316C600B8
:1036600013061611D38005F2530106F2538020226F
:10367000532500A01305F5FF63140500530500E072
:10368000B71311119B831311631275269301E00A7E
:103690009B05100093957502938515F19395C500D0
:1036A000938515119395C500938515113716F1FF74
:1036B0001B0616111316C60013061611D38005F249
:1036C000530106F253802022530500E2B713F1FFA5
:1036D0009B8313119393C300938313116318752075
:1036E0009301B0049B05100093957502938515F125
:1036F0009395C500938515119395C5009385151174
:103700001B06100013167602130616F11316C600D8
:10371000130616111316C60013061611D38005F2F0
:10372000530106F253802022532500A01305050003
:1037300063140500530500E0B71311119B831311A7
:103740006316751A9301F00A9B0510009395750294
:10375000938515F19395C500938515119395C50033
:10376000938515111B06100013167602130616F129
:103770001316C600130616111316C60013061611EB
:10378000D38005F2530106F253802022530500E254
:103790009B03100093937302938313F19393C300DD
:1037A000938313119393C3009383131163107514C0
:1037B0009301C0049B05100093957502938515F144
:1037C0009395C500938515119395C50093851511A3
:1037D000371611911B061611D38005F2530106F21C
:1037E00053802022532500A01305F5FF6314050024
:1037F000530500E0B71311119B8313116318750E65
:103800009301000B9B05100093957502938515F1AC
:103810009395C500938515119395C5009385151152
:10382000371611911B061611D38005F2530106F2CB
:1038300053802022530500E2B713F1FF9B8313113D
:103840009393C300938313116312750A9301D004F9
:103850009B05100093957502938515F19395C5000E
:10386000938515119395C500938515111B06F0FFDF
:103870001316F603D38005F2530106F2538020227B
:10388000532500A01305F5FF63140500530500E060
:10389000B71311119B831311631A75049301100B55
:1038A0009B05100093957502938515F19395C500BE
:1038B000938515119395C500938515111B06F0FF8F
:1038C0001316F603D38005F2530106F2538020222B
:1038D000530500E2B713F1FF9B8313119393C300C9
:1038E0009383131163147500631A3000139511004C
:1038F0006300050013651500730000001305100038
:0839000073000000731000C009
:083908000101010101010101AF
:10391000417373657274696F6E206661696C65646A
:103920003A2061646472203E3D202831554C203C91
:103930003C203132292026262061646472203C20FC
:103940003633202A202831554C203C3C2031322966
:103950000A00000000000000417373657274696F13
:103960006E206661696C65643A20212870745B334F
:103970005D5B616464722F2831554C203C3C2031E2
:1039800032295D2026203078303830292026262024
:103990006361757365203D3D203078660A00000044
:1039A000417373657274696F6E206661696C6564DA
:1039B0003A206E6F64650A00417373657274696FB3
:1039C0006E206661696C65643A20757365725F6D1F
:1039D000617070696E675B616464722F2831554C49
:1039E000203C3C203132295D2E61646472203D3DD3
:1039F00020300A0000000000417373657274696F23
:103A00006E206661696C65643A202122696C6C6580
:103A100067616C20696E737472756374696F6E226E
:103A20000A00000000000000417373657274696F42
:103A30006E206661696C65643A2070745B335D5B0F
:103A4000616464722F2831554C203C3C203132296E
:103A50005D20262030783034300A0000000000005D
:103A6000417373657274696F6E206661696C656419
:103A70003A2070745B335D5B616464722F2831554A
:103A80004C203C3C203132295D20262030783038D3
:103A9000300A000000000000417373657274696FA2
:103AA0006E206661696C65643A2074662D3E6570AF
:103AB0006320252034203D3D20300A000000000016
:103AC000417373657274696F6E206661696C6564B9
:103AD0003A202122756E657870656374656420658F
:103AE0007863657074696F6E220A00000000000040
:103AF000417373657274696F6E206661696C656489
:103B00003A202122756E737570706F72746564202F
:0C3B100073617470206D6F6465220A0000
:040000058000000077
:00000001FF
